:020000020000FC
:0400000006C032C044
:10000C00189548EC4DBFBB27DD27FF27EE2414D1F4
:10001C0025D1C2D0909A4CE049B9539A549A4FE0EA
:10002C0045BF40E44BBF7894B09B05C0023069F0EB
:10003C00033041F0F9CF4FEFB099F6CF4A95E1F785
:10004C00ABD0F2CF2BD304E0EFCFC0E66C2D1CD19C
:10005C009FD12AD1AFD116D204E0E6CF5FB64F9331
:10006C003F9343E032E0B09BFECFB19BFECFB19B00
:10007C0005C043E03A95000099F0F9CF32E04A957B
:10008C000000A9F707C06F90AF911F912F91CF91EE
:10009C006F91522D3F914F915FBE80E48ABF1895AE
:1000AC00252E86B36F93CF9356E06EE0CEE676B3F3
:1000BC007370A1F07795881F5A95C9F7000076B335
:1000CC00737061F07795881F57E0899386B38370BE
:1000DC0029F05A9500006A9551F7D9CFC137B8F27B
:1000EC0040916E0030916F0069F43F1559F442371E
:1000FC0011F491E0CCCF403511F493E0C8CF4E34DD
:10010C0009F40AC0483211F0463321F4913081F0E1
:10011C009330B1F090E0BBCF2F931F93AF936F92BE
:10012C000430B9F442D0EE20B1F492E003E0ABCF4E
:10013C002F931F93AF936F9286D01AD002E0A3CF68
:10014C002F931F93AF936F92023019F07CD000273E
:10015C009ACF8BD098CFFF2421E018E04F2DE79455
:10016C0008F042274795FF1C1A95C1F7EE248BCF58
:10017C00573029F05395881F5A95E9F789936C2FBE
:10018C006D56C62ECEE6A1E649914D936A95E1F7E0
:10019C0064E56093600008954AEAF42E9927992447
:1001AC00882400273324112408956D2DCFEC30E0E2
:1001BC00162F23E07991C198C09AB99AB89A48B38E
:1001CC0057E00000779508F0422748BB5A95C9F7CD
:1001DC0070FF42271A95799148BB91F7582D5030F2
:1001EC0041F0779508F0422748BB00005A95C9F7B3
:1001FC00788100004C7F48BB55E05A95F1F7C09AC6
:10020C00C09AB998B898C09808954091D0004B34D2
:10021C0043EC09F04BE44093D000089543EC409339
:10022C00D00040E84093CF00F0DF40E04093D10095
:10023C004093D20064E0089540E84093CC0042ED36
:10024C004093CD000895CF935F938F92CCEC62E0F6
:10025C008824ADDF8F905F91CF91089540E8409353
:10026C00C9004AE54093CA0008958F92C9EC62E038
:10027C0088249DDF8F90089540E84093CF004EE195
:10028C004093D00062E00895CF936F936C0F4FEFC3
:10029C0047954881242F2795242720952993C61705
:1002AC00B9F76F91CF910895112777247A94CF9352
:1002BC006F93312F48E0340F6A95E9F726E06F9180
:1002CC006F936C0F63956395488158E0479508F0E0
:1002DC0027E02A95A1F4371526E088F43A95732E79
:1002EC00513011F459E0C3955A9590FA1EF037D05D
:1002FC001A9502C01BD013956F91CF91D8CF3A9518
:10030C0021F05A9519F7C395DFCF6F91CF9190FAE1
:10031C003EF0103051F06A95185F38F46A950895E4
:10032C00812E185010F06395812E0895452F59E0B9
:10033C00541B3881331F2FEF220F5A95E9F73223C4
:10034C002095269548814223342B4881441F3993AC
:10035C00C61301C008953881331F3993F9CF452F47
:10036C0059E0541B4C2F4395C62F3A91379538833F
:10037C00C413FBCF3A9137952FEF5A9511F0220FFA
:10038C00FCCF3223209548814223342B38830895A7
:10039C00CF936F93C0E603D06F91CF9108956C0FFC
:1003AC00488138E04795221F3A95E1F72993C61703
:1003BC00B9F70895CF936F93C0E611D06F91CF9199
:1003CC000895CF936F93CFEC0AD040953095399325
:1003DC004883CA9562E0E3DF6F91CF9108956C0F6B
:1003EC00C3954991433C11F04B34A9F44FEF3FEFC7
:1003FC00299118E037FB50F95227441F331F4E7FC9
:10040C002695579520F450E8352755E045271A9541
:10041C0089F7C61769F70895C895099231966A95B8
:10042C00D9F72BC0C895099233FA36F43196C89592
:10043C000992E89433F802C0002409923196625074
:10044C0089F71BC000800992E3956A95D9F715C00E
:10045C00EEBBE09A0DB20992E3956A95C9F70DC00F
:10046C0040E84093CF0068E0C1ED332009F4D4CFCD
:10047C0032FCD8CF30FCE6CFEBCF37FC3324C5DED3
:10048C00C0ED089506D09394CFEC0EDFD62E9924B0
:10049C00089533244091620030916300407609F452
:1004AC0095C0FF27333039F1343049F1353049F1FB
:1004BC00363059F1373059F1383091F03930B1F0DC
:1004CC003A3089F13B30B9F13C3039F13D3049F1EA
:1004DC003F30D9F1E1C0F061E091640066D074C0A6
:1004EC00E091640042E0342E40E8ADC0E09164003D
:1004FC00009066004CC1609064002DD165C044D161
:10050C0007C0609064002DD15FC03BD101C02FD1DA
:10051C00E0E041E8342E41E096C04091640049B9D6
:10052C0053C009B0F5CF409164004CB9539B4CC0FB
:10053C005E9BFCCF49C05F9B66C00CB0E0E041E81D
:10054C00342E41E05B9943E07EC0F091640016D0FC
:10055C00E0937C00F091650011D0E0937E00F09167
:10056C0066000CD0E0937E00F091670007D0E0931A
:10057C007F00ECE741E8342E44E065C0EE2728E02C
:10058C0018B3EE0F46B346FBE0F9F7FB15F9187FED
:10059C0018BBC79A06D0C79804D0FF0F2A9589F7C5
:1005AC0008950000000000000895EF93E29501D03B
:1005BC00EF91EF70EF2B6E2ED4D0E0626E2ED1D077
:1005CC00EF7D6E2ECED0089541E01EC03030D9F0B4
:1005DC003130C1F03330B1F0353079F0363019F1BB
:1005EC003730F9F0383099F0393051F03A30A9F011
:1005FC003B3041F03C30A9F04FC0E09064004CC05F
:10060C001090640049C042E0F6E0E8EF1CC01120F5
:10061C00D9F241E0F6E0EFEE16C0F6E0E6EF41E08D
:10062C0012C02ADE089530916500313029F0323045
:10063C0039F03330D9F00895F6E0E8ED42E103C02B
:10064C00F6E0EAEE49E1A0906800A41608F0A42EAA
:10065C004A2DBB24477009F0B3944A2D4695469514
:10066C004695B40E43EC4093D00021C03CE0332EB1
:10067C0030916400303059F0323029F018F6F7E040
:10068C00E8E046E4E0CFF7E0ECE246E2DCCF3324EE
:10069C00F7E0E4E044E0D7CFC1DD089502D0F3DE0B
:1006AC0008954B2D413011F4BCDD0895BA943A2DC8
:1006BC00385018E018F41A2DBB24B394A32ED0DEB6
:1006CC0062E0610F7EDE639563950895120100016F
:1006DC0000000008EB030200010001020001090206
:1006EC001900010100801409040000010000000041
:1006FC000705810008000A00040309044603496E3B
:10070C00672E2049676F72204365736B6F2C2043F3
:10071C006F707972696768742863292032303033BE
:10072C00260349676F72506C75672D55534220280C
:10073C004156522960FA43F961FA45F962FA46F9D1
:10074C0063FA33F964FA34F965FA35F966FA36F96D
:10075C0067FA37F9089541B337B3ECDF41BB37BBC8
:10076C00089542B338B3E6DF42BB38BB089546B3B5
:10077C0030B333FB40F935FB41F936FB42F9042E1B
:10078C00089548B332B3F5CF47B331B3F2CFEEBBD4
:10079C000DBAF894E29A7894E19AE199FECF14CFCD
:00000001FF
